:040000000CEF00F011
:10000800E9CF0DF9EACF0EF9F3CF0FF91BEF00F0A6
:1000180000EE00F018EE2FF014EC00F07DEF05F084
:10002800EE6AE550E150FCE1E250FAE11200F4CF4B
:1000380010F9F2B6F2A02DD181CF2EF8D6CF2EF836
:10004800D7CF07F90901086BD890080119350901BC
:10005800096F08011A3509010A6F0929E96E000EAE
:100068000A21EA6E07C9EEFF08C9EDFFD89008011A
:1000780019350901076F08011A350901086F0729A1
:10008800E96E000E0821EA6EEECF09F9EDCF0AF904
:1000980009C90AF9096B08012E5109010913D890F9
:1000A8000801193509010B6F08011A3509010C6F90
:1000B8000B29E96E000E0C21EA6E09C9EEFF0AC988
:1000C800EDFF080129513DE0D89013EC05F003E35A
:1000D80008012C2B02D008012C6B0A0E2C6531D09C
:1000E8002A672FD0D89019350901076F08011A35EA
:1000F8000901086F0729E96E000E0821EA6EEECFA4
:1001080009F9EDCF0AF9650E095D190E0A5919E3C7
:10011800D890080119350901076F08011A35090136
:10012800086F0729E96E000E0821EA6EEECF01F08C
:10013800EDCF02F00801196B1A6B010E2A6FF294C9
:10014800F28A08012D5101E199D0D8901935090199
:10015800076F08011A350901086F0729E96E000EB3
:1001680008EC05F02FE3D890080119350901076F4D
:1001780008011A350901086F0729E96E000EFDEC20
:1001880004F020E2D890080119350901076F080129
:100198001A350901086FFF0E0725E96EFF0EF2EC0C
:1001A80004F010E3D890080119350901076F080118
:1001B8001A350901086FFF0E0725E96EFF0EE7ECF7
:1001C80004F03EE3D890080119350901076F0801CA
:1001D8001A350901086FFF0E0725E96EFF0E08ECB6
:1001E80005F031E3D890080119350901076F0801B6
:1001F8001A350901086FFF0E0725E96EFF0EFDECA1
:1002080004F021E2D890080119350901076F0801A7
:100218001A350901086F0729E96E000EF2EC04F09F
:1002280012E3D890080119350901076F08011A353A
:100238000901086F0729E96E000EE7EC04F003E2F4
:1002480008012C2B02D008012C6B2A670DD02B51EA
:100258000BE0D89013EC05F007E30801196B1A6B53
:10026800010E2A6FF294F28A140E08012C6506D04A
:100278002B6704D02A6702D0010E2B6F194B1A2B5B
:100288001A51020A191102E1196B1A6BD76AD66A58
:10029800F290F2BAF2A416D0F29AF294F290F29690
:1002A800F29E0801295103E09AEC02F002D0B3EC67
:1002B80003F00801196B1A6B2A6B2C6B2B6BF290ED
:1002C800F286F28E10C9F4FF0FC9F3FF0EC9EAFFD8
:1002D8000DC9E9FF110009011B6B1B51FC0DF3CF80
:1002E8001CF91C0E1C271FC81DF920C81EF921C89F
:1002F8001FF922C820F9BBEC04F01C2FFCD71D51B4
:100308000801286F010E09011B25E96EEA6A080138
:10031800080EEA2228510F0BEF6E09011B2B060E5F
:100328001B65DBD708011F510F0B086F080E090169
:100338001B6F1B51FC0DF3CF1CF93C0E1C271BC86F
:100348001DF91CC81EF91DC81FF91EC820F9BBECF1
:1003580004F01C2FFCD71D510801286F010E09015C
:100368001B25E96EEA6A0801080EEA2228510F0BDC
:10037800EF6E09011B2B0E0E1B65DBD708011B5105
:100388000F0B106F29512CE0100E09011B6F1B5128
:10039800FC0DF3CF1CF94C0E1C2723C81DF924C8EB
:1003A8001EF909011C2B03D01E351E331D331C2FCB
:1003B800FBD71D510801286F010E09011B25E96EA5
:1003C800EA6A0801080EEA2228510F0BEF6E0901AC
:1003D8001B2B120E1B65DBD7080123510F0B146F63
:1003E8002D512FE0100E09011B6F1B51FC0DF3CF8F
:1003F8001CF9540E1C2725C81DF926C81EF927C844
:100408001FF909011C29206F04D01F351F331E3323
:100418001D33202FFAD71DC928F8010E09011B2505
:10042800E96EEA6A0801080EEA2228510F0BEF6EFE
:1004380009011B2B140E1B65D8D7080125510F0B7A
:10044800166F09011B6B010E09011B25E96EEA6A8B
:10045800080EEA22EF501C6F0A0E1C5D07E21B29EA
:10046800E96EEA6A080EEA22300E08D0010E090188
:100478001B25E96EEA6A080EEA22370EEF26090103
:100488001B2B170E1B65DFD7010E32EC06F0020E90
:1004980032EC06F01B6BB1EC04F0F9EC05F0A7ECBC
:1004A80004F07FEC06F009011B2B050E1B65F3D742
:1004B800C00E32EC06F0060E1B6FB1EC04F0F9EC3E
:1004C80005F0A7EC04F07FEC06F009011B2B0F0EDA
:1004D8001B65F3D70801295113E0200EF9EC05F04C
:1004E800100E1B6FB1EC04F0F9EC05F0A7EC04F06A
:1004F8007FEC06F009011B2B130E1B65F3D710D0F8
:10050800100E09011B6FB1EC04F0F9EC05F0A7EC33
:1005180004F07FEC06F009011B2B150E1B65F3D7C1
:100528000D0E7FEC06F00A0E7FEF06F00901116B45
:10053800126B030E136F146B13A130D0D8901335C0
:10054800156F1435166F1529E96E000E1621EA6E1F
:10055800EECF17F9EDCF18F9CB0E175D0C0E185921
:1005680014E31129E96E040E1221EA6E010EEF6EF2
:10057800020E1125E96E040E1221EA6E010EEF6ECD
:10058800020E1127000E122309D01129E96E040E5C
:100598001221EA6E010EEF6E114B122B13B12DD002
:1005A800D8901335156F1435166F1529E96E000E9E
:1005B8001621EA6EEECF17F9EDCF18F9A50E175DE3
:1005C800080E185912E31129E96E040E1221EA6E79
:1005D800EF6A020E1125E96E040E1221EA6EEF6A27
:1005E800020E1127000E122308D01129E96E040EFD
:1005F8001221EA6EEF6A114B122B134B142B145174
:10060800800A7E0F000ED8B4135D96E3136B146B4B
:10061800D89008011F350901156F08012035090117
:10062800166F080121350901176F080122350901E4
:10063800186F1329E96E040E1421EA6EEF50151194
:1006480008011F6F090116510801206F0901175190
:100658000801216F090118510801226F020E0901D2
:100668001327000E14231451800A800F400ED8B4AB
:10067800135DCEE3400E136F146BD89008011B3541
:100688000901156F08011C350901166F08011D3590
:100698000901176F08011E350901186F1329E96E42
:1006A800040E1421EA6EEF50151108011B6F0901A1
:1006B800165108011C6F0901175108011D6F090126
:1006C800185108011E6F020E09011327000E14238A
:1006D8001451800A800F800ED8B4135DCEE3800ECB
:1006E800136F146B1329E96E040E1421EA6EEF5090
:1006F80023C815F924C816F9D890090115371637F3
:1007080015110801236F090116510801246F020E03
:1007180009011327000E14231451800A800FA00E1C
:10072800D8B4135DDFE308012451630AC90ED8B4B5
:10073800231913E024519C0A360ED8B423190DE06E
:100748002451410AEB0ED8B4231907E02451BE0AFC
:10075800140ED8B42319D8A412006FEF01F00901C0
:10076800116B126B020E136F146B13B124D0D89057
:10077800D5EC04F017E3C2EC04F014E21129E96E99
:10078800040E1221EA6E010EEF6E020E1125E96EBB
:10079800040E1221EA6E010EEF6E020E1127000EF2
:1007A800122309D01129E96E040E1221EA6E010EF6
:1007B800EF6E114B122B13A121D0D890D5EC04F079
:1007C80015E3C2EC04F012E21129E96E040E1221BD
:1007D800EA6EEF6A020E1125E96E040E1221EA6E26
:1007E800EF6A020E1127000E122308D01129E96EB4
:1007F800040E1221EA6EEF6A114B122B134B142BC5
:100808001451800A7E0F000ED8B4135DAEE3136B4B
:10081800146BD89008011F350901156F08012035A0
:100828000901166F080121350901176F08012235E2
:100838000901186F1329E96E040E1421EA6EEF50AE
:10084800151108011F6F090116510801206F0901D0
:1008580017510801216F090118510801226F020E72
:1008680009011327000E14231451800A800F400E2B
:10087800D8B4135DCEE3400E136F146BD890080103
:100888001B350901156F08011C350901166F080190
:100898001D350901176F08011E350901186F132945
:1008A800E96E040E1421EA6EEF50151108011B6F52
:1008B8000901165108011C6F0901175108011D6F24
:1008C8000901185108011E6F020E09011327000EB5
:1008D80014231451800A800F800ED8B4135DCEE320
:1008E800800E136F146B1329E96E040E1421EA6E3F
:1008F800EF50156F166B176B25C818F926C819F92C
:1009080027C81AF9D8900901183719371A37155115
:1009180018110801256F0901165119110801266FD0
:10092800090117511A110801276F020E090113272F
:10093800000E14231451800A800FB00ED8B4135D32
:10094800D2E36FEF01F0010E09011B25E96EEA6A97
:100958000801080EEA22EF501200010E09011B25BA
:10096800E96EEA6A0801080EEA22EF50120009014E
:10097800203520331F331E331D331200D890133512
:10098800156F1435166F1529E96E000E1621EA6EDB
:10099800EECF17F9EDCF18F9A00E175D0F0E185905
:1009A80012001335156F1435166F1529E96E000EF0
:1009B8001621EA6EEECF17F9EDCF18F9150E175D6F
:1009C800050E185912000821EA6EEECF09F9EDCF8D
:1009D8000AF9140E095D050E0A5912000821EA6E7B
:1009E800EECF09F9EDCF0AF9210E095D030E0A5978
:1009F80012000821EA6EEECF09F9EDCF0AF9580E78
:100A0800095D020E0A5912000821EA6EEECF09F9B3
:100A1800EDCF0AF92D0E095D010E0A59120019359C
:100A28000901076F08011A350901086F0729E96EDE
:100A3800000E0821EA6EEECF09F9EDCF0AF9810E12
:100A4800095D0C0E0A591200E8CFF3FF0090F36617
:100A580003D00080030E01D03F0EE96E8A908A947D
:100A68008A92939093949392946A4E0E0901006F20
:100A7800EB0EE82EFED7002FFCD7E9CF8BFF8A8438
:100A880000F000F08A941A0E0901006FF80EE82EA3
:100A9800FED7002FFCD70400E9CF8BFF8A8400F033
:100AA80000F08A94C80E0400E82EFDD7E9CF8BFF2A
:100AB8008A8400F000F08A9400A00CD062EC06F062
:100AC800020E8B6E8A8400F000F08A94280E16ECD1
:100AD80006F003D0380E16EC06F00C0E16EC06F0F5
:100AE800010E16EC06F0060E16EC06F0800E16EF58
:100AF80006F0700ED3127E6A7F6A816A826A9368F2
:100B0800946A080E7C6EF19ED09EF26AF16AF06AD1
:100B1800100E7D6E080ED56ED58EF294F29AF2867E
:100B2800F29081A605D00801296B010E2D6F04D023
:100B3800010E0801296F2D6B000E28EC05F0020E3E
:100B480016EC06F076EC06F00801196B1A6BF28EBB
:100B5800FFD70F0E946E8A8200F000F000A013D029
:100B68008A8400F000F082CF26F98A942639F00BA7
:100B7800256F8A8400F000F082CF26F98A942651E6
:100B88000F0B251308D08A8400F000F082CF26F9D5
:100B98008A9426C925F98A92946A255112000F0E63
:100BA800946E8A8200F000F000A013D08A8400F0CE
:100BB80000F082CF06F98A940639F00B056F8A8413
:100BC80000F000F082CF06F98A9406510F0B051346
:100BD80008D08A8400F000F082CF06F98A9406C90A
:100BE80005F98A92946A05511200E8CF21F94EEC72
:100BF80006F08B6A8A8000A00DD021390F0B8B126A
:100C08008A8400F000F08A94F00E8B1621510F0BA5
:100C18008B1202D021C98BFF8A8400F000F08A94DD
:100C28008A901200E8CF01F962EC06F000A00FD01C
:100C380001390F0B8B6E8A8400F000F08A94015101
:100C48000F0B8B6E8A8400F000F08A94120001C9A1
:100C58008BFF8A8400F000F08A941200E8CF21F913
:100C68004EEC06F000A00FD021390F0B8B6E8A8452
:100C780000F000F08A9421510F0B8B6E8A8400F0EB
:100C880000F08A94120021C98BFF8A8400F000F0DA
:100C98008A941200E80E0901236F030E246F2307BC
:100CA800D8A0240709012329D8B42429D8B41200CC
:100CB800ADEC05F0226F22AF1200F1D7E80E090162
:100CC800036F030E046F0307D8A004070901032963
:100CD800D8B40429D8B41200D3EC05F0026F02AFDF
:100CE8001200F1D7670EAF6E240EAC6E900EAB6E8D
:100CF800949C948E900CE8CF21F9ACA2FED721C920
:040D0800ADFF120029
:020000040030CA
:0C000000FF38F7FEFF73BBFFFFFFFFFFA0
:00000001FF
